:1000000008B5094B01221A60084B0022C360084B57
:1000100094211860074800F0DBF802F01FFF064B40
:100020004FF001121A6008BDE0930000C089000083
:10003000D4930000D88700000800074000207047D4
:100040002DE9F04FDFF85891DFF85881D9F80030EA
:1000500085B000240393C8F80040039B4E4613F07C
:10006000010F454644D0454B4FF480321A60444A54
:10007000DFF828A11368434F43F08053136000F06A
:1000800073FDDFF80CB1C0B10123CAF80030039B47
:100090003D4AC9F8003013684FF49E7043F01003D6
:1000A00013604FF00113C8F800303B68DBF8002004
:1000B0009B68D1785B6A984758E00146019002F04E
:1000C000F3FE3A68B821926840F21F10526A9047D6
:1000D000019B2E4A4FF49E7013603B68DBF80020B2
:1000E0009B68D1785B6A98470123CAF8003038E0F2
:1000F000039BDA033CD5234C40F24B1023689B68EA
:100100001B6A9847224A236812689B68527900F05C
:10011000C00111435B6A40F24B10984723684FF4CB
:100120009E709B6802215B6A98471A4B1B68DB072D
:1001300006D4236840F21F109B68B0215B6A984781
:100140000E4B002201211A60996013490B6843F499
:1001500080330B600C490B6823F010030B600F4BCE
:100160001A60039B33604FF001132B60002001E005
:100170004FF0FF3005B0BDE8F08F00BFC001084070
:1001800028300840D4930000000100408C00044057
:10019000B8890000C4120840088108400C000740DC
:1001A000040007400800074003461A46117801334F
:1001B0000029FAD1101A704710B5431EC41D0A78E1
:1001C00003F8012F02B10131A342F8D110BD0000A4
:1001D000034630B514460D4685B019466846FFF70C
:1001E000EBFF054B02951B6803949A6818689268A8
:1001F0006946904705B030BDD4930000F0B53D4B43
:100200001A68D20762D41B689B0762D43A4F3B68D6
:1002100013F4704F60D13949394A0B68394E1B0EBF
:100220001377394B08681C68B36CC0F307409D8A8C
:10023000364B25441B68696CED6DDBB2491BC31A54
:10024000B1FBF3F3A3F59C53083BB3F57A6F45D8A4
:100250003B681B0F44D12E48036882F83C30F36E94
:10026000998A2C4B0C441D68E16A636C0068C91ABA
:10027000C0F30723C3EB1563B1FBF3F3A3F59C5362
:10028000083BB3F57A6F2DD8234B196811F4704FE2
:100290002AD12249096882F85C101B681B0F26D1FD
:1002A0001F49096882F87C10D0580F2400F580514E
:1002B0008C6040F201310160D15800208860D15833
:1002C00020330124802B4C60EED1F0BD41F211109F
:1002D000F0BD42F22220F0BD0320F0BD0420F0BDAD
:1002E0003020F0BD4020F0BD4FF44070F0BD4FF421
:1002F0004050F0BD149000A0009000A01C9000A001
:10030000388900003C8F0000E8930000209000A096
:10031000289000A0249000A0049000A02C9000A0A1
:10032000309000A001234360002200F580531B6839
:1003300013F00F0306D1B2F5007F01D00132F4E7CC
:1003400018467047B2F5007F1ABF006CC0B200209B
:100350007047000070B51B4D440129194A7F1A4BA4
:100360000646242000FB02338A69DB689A4202D0E9
:100370004FF0FF3070BD2859FFF7D4FF08B32B1999
:100380001B69022E08BF00F1FF3013B1C31A062B00
:1003900016DC2B195A69B2F57A7FE9D25968013215
:1003A000814288BF58605A612B1999682C44814258
:1003B00038BF9860E3681844E060B0FBF2F0206159
:1003C000002070BD388900003C8F0000064B03EB15
:1003D00040139A6859689B7F521A9A42DDBF830086
:1003E00005209840002070473889000070B51F49EB
:1003F00001EB40110C7F4E7F14B98300062010E002
:100400001B4B1C4A1D6824237343D258938A567889
:100410004A68121B07D5511C07D0023207D083004F
:100420000720984070BD282402E03C2400E0782496
:1004300000F6283003F10C02191D800002EBC60300
:10044000046029442B44083199420CD051F8085CCF
:1004500041F66A02B5FBF4F0B0FBF2F002FB105279
:1004600041F8082CEFE7002070BD00BF388900007C
:10047000E89300003C8F000070B5214C012804EB8C
:10048000401404F118014A7901D9002070BD1D4BB8
:1004900009791D68242353431B4AD3589A8A5E78EE
:1004A0006368591A002903DC83000820984070BD56
:1004B00041F270734B4344F63E118B42A8BF0B468A
:1004C00041F66A0193FBF1F34B4300F62E318900AC
:1004D0000B60A91802EBC6022A449142D5D04C68A1
:1004E0000A4DE41A4C600C68AC4201D128B9CCE743
:1004F000074DAC4201D10128C7D00831EDE700BF5C
:1005000038890000E89300003C8F000058FC190077
:100510004811100038B50023144A02EB4312526907
:10052000F92A04D89B000E2404FA03F038BD0133E5
:10053000042BF1D10020FFF749FF04460120FFF70B
:1005400045FF044310D125462846FFF74FFF30B939
:100550002846FFF791FF10B9AB000F2098400135F6
:10056000042D44EA0004EFD1204638BD388900004C
:1005700038B5364D364A2B68934221D1354C236825
:1005800043B12368012B5ED1334B4FF400221A6034
:1005900000250DE042F6B443304A1A60012323607F
:1005A000FFF72CFE0028ECD026E00135042D19D0F1
:1005B0002846FFF7CFFE0028F7D00223236019E07A
:1005C000274A934210D0274A93420BD0912002F041
:1005D000DCFE00240120072102F066FC2C60932041
:1005E00002F0D3FE002038BD1A4B1A68012A2AD126
:1005F00002221A60FFF78EFF002422461A490D7F5F
:100600004B685B1B072B03DC13F1080F06DB00E0D4
:100610000723002D08BF6FF0070301E06FF0070309
:1006200003F00F03A3400434102C42EA030201F14B
:100630002001E4D142F6B04342EA004119600B4880
:100640000F22FFF7C5FD4FF0FF3038BD8C0004408E
:100650000000CDABD093000008000440EFBEADDE3B
:100660000100CDAB0200CDAB38890000E08700006F
:10067000013810F8012F11F8013BD31A13F0FF03D2
:1006800001D1002AF5D158B2704730B50C46451E4D
:10069000131B0B44002B04DD14F8013B05F8013F4C
:1006A000F6E730BD10B50446131B0344002B02DDF2
:1006B00004F8011BF8E710BD074BDB6ADB0009D427
:1006C00049F62033054A1860136823F07F4343EA54
:1006D00000601060704700BFD0890000AC0908407E
:1006E000124BDA6AD20020D4DB6A49F62C3113F4BB
:1006F000803F0F4A03D10F4B1B68012B09D10B68B8
:10070000C0B223F0FF0303430B60136823F0FF0321
:1007100009E00B68000280B223F47F4303430B60BF
:10072000136823F47F43184310607047D08900009A
:10073000AC090840E0930000074BDB6ADB000AD4F9
:1007400049F62833054A18601368C0B223F47F03C2
:1007500043EA004010607047D0890000AC090840AF
:100760002DE9F84F49F610331B68834603F51B4308
:10077000B3F52B4F0F4600DB30BF49F6C0339C6802
:1007800049F6E0339E6849F6F0339B68564D03F511
:100790001B4A4FF41C439B68702203F51B4949F622
:1007A00010439B6804F51B4403F51B4849F6B0331E
:1007B000996805F1600001F51B4102FB0711FFF785
:1007C00064FF04EB8711494C06F51B46402205F1F6
:1007D000D000FFF75AFF06EB4B1120224FEA471BD0
:1007E00004F1D800FFF751FF06EB0B01404E202229
:1007F00004F1F800FFF749FF0AEB0B01202206F194
:100800003400FFF742FF49463C2206F1D400FFF7CF
:100810003CFF08EB8701042206F58870FFF735FFDF
:100820004FF41B43D3E9000106F58C73C3E90001C3
:10083000304B1B68E380D6F81831C3F303132B71D8
:10084000DAB2D6F81831C3F30313D8B22374D5F84B
:10085000C830032803F0030101EA020161F3010338
:10086000C3F3011101EA020161F30513C3F301218E
:1008700001EA020161F30923C3F3013101EA020134
:1008800061F30D33C5F8C830D5F8B03003F003017B
:1008900001EA020161F30103C3F3011101EA02015C
:1008A00061F30513C3F3012101EA020161F3092396
:1008B000C3F3013102EA010262F30D33C5F8B0302F
:1008C0000FD0D4F8D8306FF38A236FF3CB23C4F85A
:1008D000D830D4F8F8306FF38A236FF3CB23C4F801
:1008E000F8300020BDE8F88F308C0000088B000045
:1008F000D0890000B4090840094B102209491A6048
:100900001A44116001F5A0215160A1F58021916088
:1009100040F221221A601A68D205FCD4704700BF49
:10092000003CA8A500000280F8B54FF490520021C9
:100930000646FFF7B7FE1C4B00221846B2F5905F43
:1009400006EB020112D0002717F0010FD0E9004595
:100950001CBFE443ED430137202FC1E9004501F1FD
:100960000801F1D102F580720830E7E70F4DAB4284
:1009700017D034460022D607D3E9000148BFC94347
:10098000F4E8026748BFC0438F4208BF864202D0E6
:1009900030BF0020F8BD0132202A2646EBD10833B3
:1009A000E5E70120F8BD00BFF08700008088000067
:1009B000C0F30723012B05D1C1F3072212B9CAB234
:1009C000052A1FD0C0F30723012B06D1C1F307234B
:1009D000112B02D1CBB2052B16D0C0F30723012B6C
:1009E00006D1C1F30723102B02D1C9B206290DD0BD
:1009F000C0F30723062B0BD0FF2B18460CBF052096
:100A00000320704718467047022070470320704744
:100A100004207047074B4FF42B4203F1100143F8B9
:100A2000042F02F50B72B2F5344F00D930BF8B4260
:100A3000F5D170471C8C000030B500F126438D00C5
:100A4000012403F59603AC401C60024B8A40C2505F
:100A500030BD00BF04004BA6C0F34070704710F0DB
:100A6000070F0CBF0120002070470000F0B51D4BA0
:100A70000022D3F8004103F58C73C4F340740128BD
:100A800013D11F68182505FB0475174995F8BD514A
:100A900051F8226005F03F05D6F8D41065F31951DE
:100AA00065F39F61C6F8D41014E0022812D11F68C4
:100AB000182505FB04750C4995F8BD5151F82260C5
:100AC00005F03F05D6F8D81065F3195165F39F611D
:100AD000C6F8D8100132042A03F10403CFD1002054
:100AE000F0BD00BF088B0000408D0000F8B51A4B28
:100AF0001A4E1B6C002513F0070F0CBF01270027AF
:100B00000024174B1B799C421EDA5CB93368154AE6
:100B100003EB471303F5F8739B68D2F838C0E8B2CB
:100B200001210CE0012C0DD1336807F1100203EB19
:100B300042130C4A9B68D2F838C0E8B202210E2258
:100B40009BB2E0470134DCE70135042D06F10406D1
:100B5000D6D10020F8BD00BFD0890000208C000055
:100B6000308C0000D88D000038B501250024064BDC
:100B7000E0B25B694FF0FF3198470134042C05EA7D
:100B80000005F4D1284638BDD88D00002DE9F04F7E
:100B900004468846174685B00193FFF73BFF204681
:100BA0004146FFF7DDFDDFF8B0C1644DDCF8002001
:100BB000DCF81010D2F8683307F0010B43F00103A2
:100BC000C1F86833D2F86423AB6C6BF310426BF35B
:100BD000C7136BF38613D8B260F30702C1F864231E
:100BE000574E584A6FF3C303136033687A1C009260
:100BF000D3F8B8309DF800A032696AF39F73C2F849
:100C0000B830514C514B04201A4602933946A36820
:100C1000CDF80CC09847029BA1461C46DDF80CC0DD
:100C2000D4F8B020DCF81030012F0BBFC3F8BC2182
:100C3000C3F8CC20D4F8C820D4F8C8200CBFC3F81F
:100C4000D821C3F8E820019AAB6C12B16BF3C7133B
:100C500002E0FF4367F3C7136FF3C3036BF386131D
:100C6000D9F8387021790D229BB20420B847EB6B7C
:100C7000D9F83870217903229BB20420B8476B6BF6
:100C8000D9F83870217901229BB20420B847AB6BA8
:100C9000D9F83870217902229BB20420B8472B6C16
:100CA000D9F8387021790B229BB20420B8476B6CBD
:100CB000D9F838700C229BB204202179B847244F10
:100CC000FB88DA0602D5FFF711FF09E01E4A1B4B2D
:100CD000946BDB6C1D4A042011799BB20E22A04755
:100CE000194A2B6D946B194A9BB211790420162274
:100CF000A047184C0420A3685146154A9847FB8822
:100D00001B0702D50098FFF7B1FE3368D7F814210E
:100D10009B680F4962F31A53326904209360656D32
:100D200043460222A847646D042002464346A44677
:100D3000074905B0BDE8F04F604700BFD08900000B
:100D4000408D0000D8930000D88D0000308C00004A
:100D5000088B0000548D0000C48D00002DE9F34184
:100D60002C4E2D4C337B4FF0000807468DF8073092
:100D70003146236886F80C8004209847274D9DF85B
:100D800007302749337304202B6898470320FFF767
:100D9000A7FCEB6A40469847EB6A01209847EB6A4C
:100DA00002209847EB6A032098470420FFF798FC3D
:100DB000236A31460420984740F2FF11AB690420B2
:100DC0009847636A042098470520FFF789FCA36AC7
:100DD000414604209847C820B847A36A012104204F
:100DE00098474FF4FA60B8470620FFF779FCE36AAA
:100DF0004146042098470120B8470720FFF770FCC0
:100E0000236B03210122042098470220B84702B037
:100E1000BDE8F081308C0000D88D0000548D0000BA
:100E2000088B00002DE9F047314D324F324C334EE4
:100E3000EB69804698472B68394604209847236819
:100E4000314600209847236831460120984723689F
:100E50003146022098473146236803209847E36AC9
:100E600000209847E36A01209847E36A02209847E8
:100E7000E36A032098472B6A394604209847A36900
:100E800040F2FF11042098476B6A04209847EB6AF0
:100E90000021042098470120C0472B6B397901229B
:100EA00004209847164E0220C0470420311806F14E
:100EB0000809636CB21D18369847A36C4946324640
:100EC00004209847EB6C49463246042098470E2090
:100ED000FFF706FC397900232C6C1A220420A04766
:100EE0000120C0476B6C39790420BDE8F0471847F2
:100EF000D88D0000308C0000548D0000088B00005D
:100F0000D08900002DE9F04100262C4DF4B26B6928
:100F100020469847EB6920464FF4802198470028E7
:100F2000264FF7DDBB6A6FF0010120469847013676
:100F300081B2BB6920469847042EE6D11320FFF703
:100F4000CFFB1F4B1F491B681F4CCB8030463B6DAE
:100F500094F831209847D4F8FC3013B10120FFF702
:100F600085FDD4F800310BB1FFF7C0FD174C2B6A9B
:100F70000420984702F026FD636D01210420984764
:100F80001920FFF7ADFB6B680E4904209847E36812
:100F90000F4904209847A36C042098470C496368C4
:100FA00004209847A36998471A20FFF799FB6369C3
:100FB00004200121BDE8F041184700BF548D000016
:100FC000B4090840088B0000D0890000D88D0000CB
:100FD000308C00002DE9F0419846274B274C1B68C8
:100FE0000F46A362264B16461B6884F83010E36256
:100FF000244B84F831209880FFF7B6FD0546002881
:1010000038D1FFF707FD94F8311094F83000FFF75E
:10101000A7FB0C20FFF764FB0D20FFF761FB4046A8
:10102000FFF700FF4046FFF76DFF1B20FFF758FB5F
:10103000154B164C1B68D3F8CC3013F4407F0FD0FF
:101040002A46384631460123FFF7A0FD02F0BAFCDC
:101050000F4BA56B1B68042003210D229BB2A847F0
:101060000C4A2369042011789847BDE8F0412020FC
:10107000FFF736BBBDE8F08120060840D0890000AC
:1010800004040840088B0000C48D0000D88D0000C7
:10109000D8930000DC930000032803D81A4B53F8C0
:1010A000203003E004282BD1174B1B685B6811F03C
:1010B000010208BF62F3410301F0020292B218BFBD
:1010C00043F0020312B143F0080301E062F3C303EB
:1010D00001F0040292B212B143F0200301E062F386
:1010E000451301F0200189B211B143F0040301E07E
:1010F00061F38203044A52F82020002053607047B5
:101100004FF0FF30704700BF408D00002DE9F04FD9
:10111000042808BF002487B008BF04940C7C18BFC3
:101120000490032C14BFA3464FF0020B049CA64D61
:1011300055F82460049C049F463455F8277051F8F4
:101140002440BF69C7F300370097049F55F8277004
:10115000BD6925F48055BD61970703D4550700F19B
:10116000BF80A8E000250595059D5D45F6D20025C8
:101170000395039D082D059D5ADC039F4FF0130C2A
:101180000CFB057504EB8505B5F84470059DDDF88D
:101190000CE04FF014080CFB05E50E3504EB85055B
:1011A0006D89DFF828E2ADB245EA0745059FDDF815
:1011B0000C9008FB07970EEB4707FF8B4FEA43099C
:1011C000BD51059D039F0CFB057504EB8505B5F826
:1011D00020A0059D4D4404EB450595F84751019528
:1011E000059D2F46039D0CFB0755063504EB850531
:1011F000B5F806C0059D9DF90470A94409F1A00940
:1012000004EB490999F80650BA441FFA8CFC6FB2F6
:10121000BC44059D4CEA0A47DDF80CC008FB05C834
:101220000EEB480EBEF80C50AF51039D01359FE701
:101230004FF04C0A0AFB054595F869E0059DDFF87B
:101240008CC10AFB054560352D7A059F45EA0E2EB7
:10125000282507FB055767443F894FEA430846F8AE
:1012600007E0059F0AFB074797F86790059F4744EB
:1012700004EB470797F847E1059F4FFA8EFE0AFBFC
:10128000074797F866A0059FF1444744A03704EB51
:10129000470797F80680DDF814E04FFA88F70EFB51
:1012A0000555AC44BCF80A50BA444AEA09277751BC
:1012B000059D013557E7049D434C009E54F8255089
:1012C000AC6924F4805444EA0634AC61049C0134D3
:1012D00084420494FFF62AAF002007B0BDE8F08FE7
:1012E00000250595059D5D45E5D200250395039DE7
:1012F000082D059D65DC039F4FF0120E0EFB057552
:1013000004EB8505B5F8B880059D4FEA43094D44C7
:1013100004EB450595F87B71059DDDF80CC07FB2A7
:101320000EFB05C52C3504EB8505B5F806C0059DFB
:10133000B8444D44BC3504EB4505AD781FFA8CFC30
:101340006FB2BC44059D4CEA0847DDF80CC0DFF8DD
:101350007C800EFB05C508EB4505B5F85C50AF5128
:10136000059D039F0EFB057504EB8505B5F8DCA014
:10137000059D4D4404EB450595F87BC1059F039DF4
:101380004FFA8CFC0EFB0757343704EB87077F8935
:10139000059DBFB24D44BC3504EB4505AD78E24434
:1013A0006DB22F44059DDDF80CC047EA0A470EFBDD
:1013B00005CE08EB4E08B8F86E50AF51039D0135CD
:1013C00094E701358DE700BF408D00008088000064
:1013D00004282DE9F74F18BF804681460F469346F3
:1013E00008BF4FF0000808F14504A300754C01EB5D
:1013F000030A1C4425685AF8046FAB69C3F3003331
:101400000193AB6923F48053AB61D5F8B43043F456
:101410000013C5F8B430D5F8B4303288C3F31503DF
:1014200043EA8253C5F8B430D5F8B43023F400133E
:10143000C5F8B430FB88990641BFB378EB67B37940
:10144000C5F8803044BFB37AC5F88430FB885A06AB
:101450001ED52268136943F0800313612268536824
:1014600043F001035360D6F80E30EB6623689A6FA1
:1014700042F001029A679A6F22F001029A675A6855
:1014800022F001025A602268136923F0800313617D
:10149000FB88DB0726D52268536843F002035360BC
:1014A0002268136943F480631361B28A738A43EA42
:1014B0000243C5F8F030F27DB37D43EA0223C5F85C
:1014C000FC30728B338B43EA0243C5F8E435727FFC
:1014D000337F43EA0223C5F8F0352268136923F409
:1014E00080631361FB88980714D522680420536831
:1014F000394643F0080353602268136943F480734C
:10150000136102225B46FFF701FE2268136923F490
:1015100080731361FB88590714D52268042053682F
:10152000394643F0200353602268136943F4007383
:10153000136102465B46FFF7E9FD2268136923F455
:1015400000731361FB881A0614D53B7C012B11D163
:101550002268136943F040031361B6F9B021B6F96C
:10156000AE3143EA0243C5F894362268136923F08A
:1015700040031361FB88DB0511D52268136943F032
:1015800040031361B6F9B821B6F9B63143EA024314
:10159000C5F898362268136923F04003136154F8A4
:1015A000042B0199936908F1010823F4805343EA5D
:1015B0000133C8459361FFF61DAF002003B0BDE8BD
:1015C000F08F00BF2C8C0000032803D80B4B53F87E
:1015D000203003E004280DD1084B1B68074A1B6D1F
:1015E00052F8202043F0807313656FF3186313657E
:1015F000002070474FF0FF30704700BF408D000063
:10160000032803D80E4B53F8203003E0042814D1EC
:101610000B4B1B680A4AD3F8B03052F8202043F035
:101620002003C2F8B0306FF38613C2F8B03043F035
:101630004003C2F8B030002070474FF0FF307047D1
:10164000408D0000032803D80C4B53F8203003E0F2
:10165000042810D1094B1B68084AD3F8B03052F85F
:10166000202061F31123C2F8B0306FF34513C2F8A4
:10167000B030002070474FF0FF307047408D0000C1
:10168000032803D80A4B53F8203006E0042802D080
:101690004FF0FF307047064B1B68D3F8B020D3F8EB
:1016A000B4305006F4D59206F2D501EA0300704733
:1016B000408D0000032803D8134B53F8203006E078
:1016C000042802D04FF0FF3070470F4B1B684A1CB4
:1016D000D3F8B03006D10C4B53F82030D3F8B40017
:1016E000800D70470231EDD1074A43F4000352F8F0
:1016F0002020C2F8B030D2F8B4006FF3D753C2F84C
:10170000B030C0F309207047408D0000032830B589
:1017100003D84A4B53F8202006E0042802D04FF0AB
:10172000FF3030BD454B1A68D2F8C833D2F8CC131D
:10173000D2F8D043072262F30F04404A43F000631B
:1017400052F8201043F48023C1F8D043012464F3FD
:101750008303C1F8C833042843F00203C1F8C83337
:1017600014D11468D4F8CC13C907FBD55468D4F845
:10177000CC13CD07FBD59468D4F8CC13C907FBD59F
:10178000D468D4F8CC13CD07FBD503E0D1F8CC4313
:10179000E407FBD552F820406FF34103C4F8C83387
:1017A00003286FF39243C4F8C83303D90428B6D191
:1017B000224B1C68D4F8C833D4F8CC13D4F8D043E7
:1017C00052F8204043F48023C1F3C205C4F8C83363
:1017D000C1F3821165F3D13361F30E336FF38303E9
:1017E000C4F8C833042843F00203C4F8C83315D141
:1017F00012490C68D4F8CC13C907FBD55468D4F847
:10180000CC13CD07FBD59468D4F8CC13C907FBD50E
:10181000D468D4F8CC13CD07FBD503E0D4F8CC13AF
:10182000C907FBD552F820206FF34103C2F8C83333
:101830006FF39243C2F8C833002030BD408D0000E2
:1018400010B50C780023497864F30F2361F3070384
:101850001178527861F31F6362F31743024A52F81A
:101860002020C2F8AC3010BD408D0000F0B54C789F
:101870000B78002743EA042363F31F47CC788B7867
:10188000002643EA042363F30F074C790B79002504
:1018900043EA042363F31F46CC798B7991F80FE078
:1018A00043EA042363F30F064C7A0B7A43EA0423DA
:1018B00063F31F45CC7A8B7A43EA042363F30F0565
:1018C0004C7B0B7B43EA0423002463F31F448B7B94
:1018D00043EA0E2363F30F04537803F001011378F6
:1018E00003F0010343EA4103002163F38F31D3780E
:1018F00003F0010E937803F0010343EA4E0363F310
:101900000D31537903F0010E137903F0010343EA1B
:101910004E0363F38B21D37903F0010E937903F027
:10192000010343EA4E0363F30921537A03F0010EE6
:10193000137A03F0010343EA4E0363F38711D37A6A
:1019400003F0010E937A03F0010343EA4E0363F3BD
:101950000511537B03F0010E137B03F0010343EAEF
:101960004E0363F38301D37B03F0010E937B03F0FB
:10197000010343EA4E0363F30101164B53F8203091
:10198000C3F89870C3F89C60C3F8A050C3F8A44093
:10199000C3F8A810C3F83C79C3F84069C3F84459A8
:1019A000C3F84849C3F86C19C3F84C79C3F85069B7
:1019B000C3F85459C3F85849C3F87019C3F85C798F
:1019C000C3F86069C3F86459C3F86849C3F8741967
:1019D000F0BD00BF408D000070B50446264891F868
:1019E00026500268042C536843F4800365F39A631D
:1019F00050F8245043F000636B60936891F82750CF
:101A000065F31343D1F8145165F31A5350F8245079
:101A1000AB6093694D7E50F8240065F3CF338D7E23
:101A200065F38E33CD7E65F34D330D7F65F30C3357
:101A30004D7F65F3CB2318BF25468361D2F8B830BC
:101A400091F82C2008BF002562F34D33C0F8B83060
:101A5000EEB23046FFF7D4FD30464FF48021FFF759
:101A60000FFE0028F8DD30460135FFF7ADFDA54239
:101A7000EEDB002070BD00BF408D00000F4BD1F8A1
:101A8000F82053F82030C3F8BC20D1F8FC20C3F86C
:101A9000C420D1F80021C3F8CC20D1F80421C3F828
:101AA000D420D1F80821C3F8DC20D1F80C21C3F8E8
:101AB0003429D1F81021C3F8002A7047408D000066
:101AC000012910B503D11146FFF7D8FF20E0022904
:101AD0001ED1104BD2F8F81053F82030C3F8C010C4
:101AE000D2F8FC10C3F8C810D2F80011C3F8D01017
:101AF000D2F80411C3F8D810D2F80811C3F8E010D6
:101B0000D2F80C11C3F83819D2F81021C3F8042AFE
:101B1000002010BD408D00000328F8B506460C4695
:101B200001D8074603E0042840F090810027C94D02
:101B3000627C55F827301B6862F39F73A27C62F3C6
:101B40001D73E27C62F3DB6343F04073227D6FF32D
:101B5000575362F31453627D62F3D343A27D62F361
:101B60008E33E27D62F30D23227E62F3C713D4F835
:101B7000E020C2F3807262F39A63D4F8D820C2F3F3
:101B8000403262F3CF33D4F8E020D20F62F38613F1
:101B9000D4F8D820C2F3853262F3050355F8262025
:101BA0001360237C012B0BD155F82730DB69C3F37D
:101BB000006262F3196355F826206FF30D33D36189
:101BC00055F827108B69D4F8E02043F48043C2F322
:101BD000016262F3010355F826209361D1F8B03019
:101BE000D4F8DC00C0F3807060F30003D4F8DC00AC
:101BF000C0F3074060F31F63C2F8B0304B68D4F8FD
:101C0000D8106FF39653C1F3802161F31C73D4F89D
:101C1000D810C1F3C02161F35D73D4F8D810C1F3BB
:101C2000402161F3D753536055F8273094F82820AA
:101C30009B6862F30603D4F8EC2062F3CD1355F8E9
:101C40002620936055F82730DB68D4F8EC20C2F3E7
:101C5000C02262F31C73D4F8E020C2F3407262F336
:101C60009E73D4F8E020C2F3033262F31B63D4F80E
:101C7000E020C2F3032262F31753D4F8E020C2F34A
:101C8000031262F31343D4F8E02062F30F33D4F865
:101C9000D820C2F3003262F3DF73D4F8E020C2F33D
:101CA000004262F35D7355F82620D36055F8273063
:101CB0001B69D4F8D820C2F3002262F3CB2355F875
:101CC0002620136155F8271094F82B204B6962F3F6
:101CD000050394F8292062F38A1394F82A2062F30A
:101CE000CB23D4F8EC20C2F3074262F31F6355F80C
:101CF00026205361D1F8C803D1F8D423D1F8E033BA
:101D0000D1F8ECC3D4F8E4E040F00040CEF3C23E9A
:101D10006FF314506EF31A60D4F8E4E0CEF3023E91
:101D20006EF31E70D4F8F0E0CEF3C24E6EF3D542DF
:101D3000D4F8F0E0CEF3024E6EF31242D4F8E4E0B1
:101D4000CEF3C20E6EF3C502D4F8E4E06EF30202E5
:101D5000D4F8E8E0CEF3024E6EF3C503D4F8E8E021
:101D60001EF4E02FD4F8E4E008BF43F00203CEF302
:101D7000422E6EF3CD22D4F8E4E018BF6FF3410396
:101D8000CEF3821E6EF30A22D4F8E8E043F001039A
:101D9000CEF3C24E6FF382036EF3CD23D4F808E185
:101DA0001EF4601FD4F8E4E008BF43F40073CEF3E0
:101DB000055E6EF3050CD4F8E4E018BF6FF3492319
:101DC0004FEA9E6E6EF30D2C43F4807355F826E0B7
:101DD0006FF38A23CEF8C803CEF8D423CEF8E033CD
:101DE000CEF8ECC3D1F80034D4F8F0203046C2F37A
:101DF000013262F38F33D4F8F0202146C2F38122FE
:101E000062F30D33D4F8F020C2F3012262F3092308
:101E1000D4F8F02062F30303D4F8F020C2F30312E5
:101E200062F30713CEF80034FFF728FE55F8273089
:101E3000A288D3F8B830002062F30B03012262F3CA
:101E40009F7355F82620C2F8B830F8BD4FF0FF3028
:101E5000F8BD00BF408D0000042870B54FF00003AE
:101E60004CD81C46072A61F31D744FF0090161F339
:101E7000195414D98A4205D00A2A05D0082A05D156
:101E8000102304E0082302E0042300E030BF43F005
:101E9000020300216FF300036FF311010FE063F3FE
:101EA00004136FF3C30301216FF3820301FA02F2FB
:101EB00043F0020300216FF3000362F31101114AA2
:101EC000102552F820606FF30005346052F820406E
:101ED000A363A16052F820305D6011684B68002B4D
:101EE000FCD151684B68002BFCD191684B68002BEA
:101EF000FCD1D36858680028FCD170BD4FF0FF308A
:101F000070BD00BFC48D000010B503289FBF0A4BF1
:101F1000002461F31D7462F319549FBF53F820200D
:101F20000121146053F820209DBF516053F82030E8
:101F3000D8684FF0FF3010BDC48D0000032810B5E5
:101F40000AD8194B012953F820309A6A104610D14B
:101F500042F48030986208E004280DD1124B012928
:101F60001C68A26A104604D109E09A6AD203FCD523
:101F700018E0C0F3004010BD4FF0FF3010BD42F438
:101F800080301A699062A26AD203FCD559688A6AC5
:101F9000D403FCD599688A6AD003FCD5DA68936AC1
:101FA000D903FCD5012010BDC48D00000328F0B575
:101FB00003D8174B53F8203003E0042824D1144BE6
:101FC0001B689A6A124B42F0010253F82010042851
:101FD0008A620FD193E8E000DC68A96A8907FCD522
:101FE000B16A8907F9D5B96A8907F6D5A16A89075F
:101FF000F3D502E08C6AA407FCD553F820306FF3C8
:1020000000029A620120F0BD4FF0FF30F0BD00BF2A
:10201000C48D0000032803D80E4B53F8203003E092
:10202000042813D10B4B1B684A79D3F8803262F332
:1020300017438A7962F30F23CA7962F30103054AD1
:1020400052F820200120C2F8803270474FF0FF3054
:10205000704700BFC48D0000032803D80E4B53F80F
:10206000203003E0042813D10B4B1B689B6A0A4AFB
:1020700039B952F8202061F30C33936243F4805352
:1020800003E052F820206FF30C3393620020704776
:102090004FF0FF30704700BFC48D0000032803D805
:1020A0000C4B53F8203003E0042810D1094B1B6877
:1020B0004A1C18BF074A9B6A1BBF52F8202061F3D5
:1020C0000413C3F30010936218BF002070474FF051
:1020D000FF307047C48D0000032810B503D80C4BA7
:1020E00053F8203003E004280FD1094B1B68084C3B
:1020F0005B6A54F820006FF30003436261F3051339
:1021000062F300034362002010BD4FF0FF3010BDAA
:10211000C48D0000032803D80E4B53F8203003E091
:10212000042814D10B4B1B6891F853205B6C62F3AD
:10213000C30391F8522062F3820391F84F2062F3B7
:102140004103044A52F820200120536470474FF0A5
:10215000FF307047C48D000063F39E7202F00303EA
:102160000B4063F30102C2F301130B4063F305124A
:10217000C2F301231940174B61F3092253F82010D1
:102180000328C1F800236FF3DF72C1F8002342F087
:102190000042C1F8002304D8D1F804331807FBD556
:1021A00013E01868D0F804231207FBD55868D0F85C
:1021B00004231207FBD59868D0F804231207FBD537
:1021C000DA68D2F804331B07FBD50022C1F80023DC
:1021D000704700BFC48D000070B54C780B78CD7887
:1021E00043EA0423002463F30F048B78CE7943EA97
:1021F000052363F31F444D790B7943EA052500233A
:1022000065F30F038D7945EA062565F31F433D4DC0
:1022100055F82000C0F81043C0F814334C7A0B7AFC
:10222000CD7A43EA0423002463F30F048B7A43EA54
:10223000052363F31F444D7B0B7B43EA05250023F5
:1022400065F30F03CD7B897BC0F8404341EA05214C
:1022500061F31F43C0F844335178137801F0010152
:1022600003F0010343EA4101002361F30103D17844
:1022700001F00104917801F0010141EA440161F3A8
:102280000513517901F00104117901F0010141EACE
:10229000440161F30923D17901F00104917901F03E
:1022A000010141EA440161F30D33517A01F0010467
:1022B000117A01F0010141EA440161F31143D17A3D
:1022C00001F00104917A01F0010141EA440161F356
:1022D0001553517B01F00104117B01F0010141EA2A
:1022E000440161F31963D17B927B01F0010102F09B
:1022F000010242EA410262F31D73C0F81833002064
:1023000070BD00BFC48D0000024B01221A60002284
:102310001A6070470011A2A5024B1A68D207FCD4BC
:10232000704700BF0411A2A5032803D80F4B53F830
:10233000203003E0042816D10C4B1B68D3F8383248
:10234000C3F3401211B16FF3451301E043F02003D2
:10235000064951F820100020C1F8383282F00103FC
:10236000034A136070474FF0FF307047C48D000080
:10237000DC93000010B5544B012902BF53F82040F4
:10238000F03443F8204053F82030146E01299C6546
:10239000546EDC65946E1C66D46E5C66146F9C662D
:1023A000546FDC66946F1C67D46F5C67D2F8804012
:1023B0009C67D2F88440DC67D2F88840C3F8884034
:1023C000D2F88C40C3F88C40D2F89040C3F89C40BF
:1023D000D2F89440C3F8A440D2F89840C3F8A8407B
:1023E000D2F89C40C3F8B840D2F8A040C3F8BC4033
:1023F000D2F8A440C3F8C040D2F8A840C3F8C44003
:10240000D2F8AC40C3F8C840D2F8B440C3F8D040CA
:10241000D2F8B840C3F8D440D2F8BC40C3F8D84092
:10242000D2F8C040C3F8E040D2F8C440C3F8E4405A
:10243000D2F8CC40C3F8EC40D2F8D040C3F8F84012
:10244000D2F8D440C3F8FC40D2F8D840C3F80041D9
:10245000D2F8DC40C3F80441D2F8E040C3F80841A8
:10246000D2F8E440C3F80C41D2F8E840C3F8104178
:10247000D2F8EC40C3F81441D2F8F040C3F8184148
:10248000D2F8F440C3F81C41D2F8F840C3F8204118
:10249000D2F8FC40C3F82441D2F80041C3F82841E7
:1024A000D2F80441C3F82C41D2F80841C3F83041B6
:1024B000D2F80C21C3F8342102BF034AF03B42F8A2
:1024C0002030002010BD00BFC48D000000000000BF
:1024D000F8B50C460546344B22469B6800219847C8
:1024E000324B302253F82530C3F83822217A0022AB
:1024F00061F35962617A61F31862A17A61F34D3236
:10250000E17A61F30C32217B61F34102617B61F37B
:1025100000021A64A17B002261F3C3022449D1E9BD
:1025200000671FA1D1E900018F4208BF8642E17B0D
:1025300008BF42F0080261F38202217C002061F3AF
:102540004102617C61F300029A646269C3F860220F
:10255000A269C3F86422E269C3F84822226AC3F878
:102560004C22626AC3F85022A26AC3F85422E26A7B
:10257000C3F85822226BC3F86822626BC3F870223A
:10258000A26BC3F87822E26BC3F86C22226CC3F80A
:102590007422626CC3F87C22F8BD00BFAFF30080E8
:1025A0003201303006000000D88D0000C48D0000DC
:1025B000E88A000070B591F848200646022A0C46C9
:1025C0004FF0000305D10979012902D161F31963A4
:1025D00001E062F3196394F849201F4D62F30F2361
:1025E00094F84A20304662F3861394F84B20002179
:1025F00062F3451394F84C2062F3041394F84D20D1
:1026000062F3C30394F84E2062F3000355F82620CA
:10261000C2F83832FFF788FE94F85F20002362F397
:102620001B6394F85D2062F34E333AB994F85C2052
:1026300062F3134394F85E2062F30C3355F82620BE
:102640000020D364D4F8C830C2F8E830D4F8B030F1
:10265000C2F8CC3070BD00BFC48D0000042830B576
:1026600028D8DBB2002563F31105144B002461F375
:102670001D7453F8201062F319540C6053F82010A5
:1026800016248C638D6053F8201010226FF3000223
:102690004A6019684A68002AFCD159684A68002AC9
:1026A000FCD199684A68002AFCD1DB685868002888
:1026B000FCD130BD4FF0FF3030BD00BFC48D0000F5
:1026C000032870B503D81C4C54F8205003E00428AC
:1026D0002FD1194C25682C6D6E6D44F4800462F383
:1026E0000406154A6FF3145452F8205061F319642C
:1026F00063F311446E6504282C6544F480142C6542
:1027000011D192E83200D3680A6DD602FCD4226D52
:10271000D002F9D42A6DD202F6D4186DC0F300505D
:102720000028F1D170BD286DC0F300500028FAD107
:1027300070BD4FF0FF3070BDC48D0000032803D87A
:102740001A4B53F8203003E004282BD1174B1B6899
:102750001B6D164A6FF396536FF3145361F31963AD
:1027600052F8201004280B6543F480130B651346C0
:1027700012D111680A6DD202FCD459680A6DD002D8
:10278000FCD499680A6DD202FCD4DB68186DC0F3E2
:1027900000500028FAD17047086DC0F3005000289F
:1027A000FAD170474FF0FF30704700BFC48D000072
:1027B000032803D8154B53F8203003E0042821D117
:1027C000124B1B681A6A114B42F0010253F8201099
:1027D00004280A6211D119680A6AD207FCD4596820
:1027E0000A6AD007FCD499680A6AD207FCD4DB686D
:1027F000186A10F00100FBD17047086A10F0010060
:10280000FBD170474FF0FF30704700BFC48D000010
:102810000346406918B1024A597E52681047704712
:102820005C8E00000346406918B1024A997E5268E6
:10283000104770475C8E0000814238BF014638B5B2
:102840001546127E002494422B6905DA53F83400B1
:10285000814202D20134F6E7013C686810B9286869
:1028600068B908E00B4A03EBC4035268D988904763
:102870000028F4D038BD2B6953F8340038BD2B69DB
:10288000054A03EBC4035268998890470028F2D0A8
:1028900038BD00BF648E00005C8E000010B5044699
:1028A000806810B9E06830B910BD064B5B68984786
:1028B0000028F7D010BD044B01215B68BDE8104033
:1028C000184700BF508E00005C8E000010B5044613
:1028D000C06810B9606850B906E00B4B00215B6816
:1028E00098470028F6D010BDA06838B910BD074B36
:1028F00001215B6898470028F6D010BD044BBDE865
:1029000010409B68184700BF5C8E0000648E00007A
:10291000508E00002DE9F74F0E9D92460F9A9B4670
:10292000954280460D9B109C0AD003FB00F94B4357
:10293000019302E088424ED301350F9B9D4201D3A3
:10294000002077E03BF81560B8F1000F06F00303B4
:102950003AF8132026F0030343EA024704DB0C9BFA
:1029600003EB0902505D1EE0B4F1007F12D009D8DC
:10297000B4F1807F16D1314A1068314A304412696F
:10298000904710E0B4F1407F06D0B4F1806F09D1D8
:102990002C4A02E02C4A00E02C4A12683846904744
:1029A000C0B200E0FF200C9B019A9A18119B515D68
:1029B000032BC1D801A252F823F000BF35610000FB
:1029C000CD610000D3610000D7610000884202D8C9
:1029D000B2E78842B0D0B4F1007F01D11A4A04E0D6
:1029E00007D9B4F1407F1AD1184A52683846904747
:1029F00012E0B4F1807F9FD1104B114F1B681E4431
:102A00003046FB689847A8B93B683046984701288C
:102A100092D07B683046984700288DD00AE0B4F108
:102A2000806F89D1074A09B1526800E09268384640
:102A30009047F1E703B0BDE8F08F00BFE8930000D6
:102A40003C8E0000508E00005C8E0000648E000002
:102A500030B50B6808495A7809689C8A002393426C
:102A600006DA0D1955F83350854203D90133F6E7DC
:102A70004FF0FF33184630BDE89300002DE9F04FCA
:102A800093468FB00E461D999DF860200A911E99BD
:102A90009DF864400D910BEB03010B461344099321
:102AA000002A08BF0B46089323440C930A9B1AAFD5
:102AB0000A44054697E880030B910791144433B10B
:102AC0000D9B13F1000A18BF4FF0010A01E0DDF879
:102AD00028A0089BCDF8009002930C9B01940393CF
:102AE0004FF08063049300230593284631463A460D
:102AF0004346FFF70FFF002840F08380079B0590B7
:102B00000293099BCDF8009003934FF04073049318
:102B10000194284631463A464346FFF7FBFE00281B
:102B20006FD1BAF1000F68D14FF080730493CDF8E4
:102B300000900194CDF808A0CDF80CB0CDF814A009
:102B4000284631463A464346FFF7E4FE002858D16E
:102B50000B9BCDF8009003934FF000730493022376
:102B600005930194CDF808B0284631463A464346CD
:102B7000FFF7D0FE002844D1BAF1000F29D0079BFF
:102B80004FF0010A0293099BCDF8009003934FF098
:102B9000407304930194CDF814A0284631463A4678
:102BA0004346FFF7B7FE60BB089B28461A930C9B71
:102BB00031461B934FF080631C933A464346CDF851
:102BC00060901994CDF874A00FB0BDE8F04FFFF7F6
:102BD000A1BE4FF08073049301230593CDF80090BC
:102BE0000194CDF808A0CDF80CB0284631463A46FD
:102BF0004346FFF78FFE20B9C1E70D980A9B98471F
:102C0000A6E70FB0BDE8F08F10B588B09DF828405A
:102C100000949DF82C4001940C9C02940D9C03940C
:102C20000E9C0494002405940694FFF727FF08B037
:102C300010BD00002DE9F04F894614468246DFF8AA
:102C4000E881517AD8F8003091B0D2F800B00C93F6
:102C500000220123704849EA01710F93BBF81470F8
:102C6000FDF7B6FA21465046FFF7F2FE214606462A
:102C70004846FFF7EDFE8642054600F0C380002E71
:102C8000C0F2C2800028C0F2BF80637A07EBC5079C
:102C90000A93237A0993614B09985A690D939047D7
:102CA0000C9B22693B445F680B901744B8420D9B14
:102CB00006D8D3F810C0099839460A9A0FABE047F6
:102CC0006268002A00F08280137E002B7ED050467E
:102CD0004946FFF7B1FD031EC0F29A802146FFF777
:102CE000B7FE81466068FFF7D9FD002840F08F806D
:102CF0009BF80510DFF830A19BF80320DAF800E01C
:102D00009BF8043000919BF809100BF10C0801911D
:102D1000CDF80880BBF8120070440390BBF8161081
:102D20003046714404913E490591616806914946D7
:102D3000FFF7A4FE00286AD1DAF80030BBF81620AD
:102D4000BBF812E01A4400929BF802200290019214
:102D50009BF80320304603924FF0807204920222C7
:102D60000592294642467344FFF7D4FD00284ED110
:102D70009BF80510DAF800609BF803209BF80430FC
:102D800000919BF80910CDF808800191BBF8120062
:102D900030440390BBF81610484631440491214951
:102DA0000591616806912946FFF768FE78BB606867
:102DB000FFF78CFD58BB0B9BBB4223D9174B0998DF
:102DC0001C6939460A9A0FABA0471BE09BF8051017
:102DD000D8F800409BF803209BF8043000919BF842
:102DE000091001910BF10C010291BBF81200204473
:102DF0000390BBF816103046214404912946FFF792
:102E000003FFD7E7002303E04FF0FF3300E0034662
:102E1000184611B0BDE8F08FE8870000A4930000C9
:102E20001160000025600000E893000010B5036801
:102E3000094A58789B8A126804331344002282425C
:102E400003F1080306DA53F8084C01320C4443F846
:102E5000084CF4E710BD00BFE893000010B500F087
:102E6000B5F901F0BFFCBDE81040014B1B681847E5
:102E7000A493000010B513680068022B096807D0FE
:102E8000032B08D053B9BDE81040064B1B68184708
:102E9000044BDB6801E0034B1B6998474FF0FF30A0
:102EA00010BD00BF248F000038B504460D46AC426B
:102EB00010DC094B20465B69984758B1036A3BB167
:102EC0009847024620B105482146002300F008F843
:102ED0000134ECE738BD00BF248F000030000080D3
:102EE000704700207047002070470020704700683E
:102EF00080B27047036889B21B0C1B040B4303604C
:102F0000036813F48033FBD11846704700207047E4
:102F1000002070470020704703681868C00F704792
:102F200030B50368C4881B68002B01DBE0B230BDFC
:102F3000064904301940002293B2A34204D250F84B
:102F4000045F01328D42F7D1D8B230BD073FFF0395
:102F5000214B10B5984204460A460BD003F5801366
:102F6000984207D01D4B1B6803F19C5303F58073F7
:102F7000984227D1236823F0100141EA0211216011
:102F80000021206810F0800F154803D0814203D043
:102F90000131F6E781421DD112482146C3F30013E7
:102FA0000CE0814207D00131206810F4803F0C48CA
:102FB000F7D181420ED121460A489BB2BDE81040AC
:102FC000FFF78EBF036889B2180C0004014321602B
:102FD0000021E9E7002010BD000180A6B88E0000A6
:102FE000A0860100100000800B46F0B5C2880446A0
:102FF00093420168868800F1080004D311462E48E8
:103000001A46002352E00A6822F010020A608D6816
:1030100025F0405222F0030242F002028A6050F88A
:1030200023000B68C0F3052E002B0BDA00230F687A
:1030300017F0005F214F03D1BB4222D00133F6E7E6
:10304000BB421ED00B6823F000430B60962303FBAA
:103050000EF20B0C1B049A510B68194A1A40194BBB
:1030600042F0004203401A430A600023086810F04F
:10307000005F124803D1834203D00133F6E7834255
:1030800001D1114811E00A68002342F010020A60E1
:1030900008680A4E10F0800003D0B34203D0013319
:1030A000F6E7B34206D108482168044BBDE8F0407A
:1030B000FFF716BF8D60F0BD17000080A0860100ED
:1030C000F8C000FC073FFF031400008030B5044641
:1030D000036800211A6822F010021A6018680B4D6C
:1030E00010F0800003D0A94203D00131F6E7A942D5
:1030F00006D121680648054BBDE83040FFF7F0BE19
:103100001A6822F000421A6030BD00BFA08601009C
:103110001300008030B50446016800230A6842F0BD
:10312000004242F010020A60086810F0005F0E488A
:1031300003D183420FD00133F6E783420BD0002343
:103140000868094D10F0800003D0AB4203D0013372
:10315000F6E7AB4206D121680448034BBDE8304096
:10316000FFF7BEBE30BD00BFA08601001200008088
:103170000A4B98420BD003F58013984207D0084BB6
:103180001B6803F19C5303F58073984203D10068D8
:10319000C0F300107047006880B27047000180A63D
:1031A000B88E000081B10123002902DB49005B00D9
:1031B000FAE7002233B181429CBF401AD218490875
:1031C0005B08F7E7104670470846704700207047D5
:1031D00009289DBF024B242202FB003000207047CB
:1031E0003C8F00002DE9F341154D01232424019368
:1031F00004FB00531F7A19B146F2A8121A6100E0CD
:103200001961444305EB04081946D8F80C00FFF790
:103210001FFC2B590B4A9B8A126803EBC000104419
:103220004368D8F81010084A19441469384698F8C9
:10323000092001ABA047002002B0BDE8F08100BF2B
:103240003C8F0000E8930000A49300002DE9F74FA5
:103250000C463C4924260228804606FB00161FD156
:10326000394B3A4D1F682A683948019239493A4A20
:1032700027F0010CD0F80090D1F800A0D2F800B0EF
:10328000C3F800C0019B23F001032B6029F0010566
:1032900005602AF0010008602BF00101116018E0C0
:1032A000042816D12D4A944207D12D4A40F61A70AF
:1032B0001268F8219268526A0AE0D1F89C10914293
:1032C00007D140F61A70264AFA2112689268526AAB
:1032D00090471C4D242202FB08525369083223B147
:1032E000516830462246984704E0506821463246ED
:1032F000FFF7A0FC0646E8B9242202FB0852B8F109
:10330000020FD4601AD1104A1760019B02F5806247
:103310001360C2F80094C2F800A8C2F800BC6EB1F5
:10332000242202FB08554146EA6823460D48FFF770
:10333000D7FD03E0B8F1020FF2D1E4E7304603B065
:10334000BDE8F08F3C8F0000000084A6000484A636
:10335000000884A6000C84A6001084A6D05408009F
:10336000D493000020000080024B242202FB003096
:10337000FFF75CBD3C8F0000036843F0100303605F
:10338000704703689B00FCD5704700F58070FDF71F
:10339000A7B910B501249C40914204D80B5823438F
:1033A0000B500431F8E7002010BD00002DE9F0417A
:1033B0002D4B2E4F93F8985086B07B6A284698473D
:1033C00080464FF49870FDF78BF9002401238DE8B7
:1033D0001800274B21460293264B22460393264B87
:1033E0004FF0FF3004932346FFF70EFC064640F2F1
:1033F0003110FDF775F97B692846D8F82480984785
:10340000C0471E4A1E4D136840F2331043F01003AC
:103410001360FDF765F929681A4A1B488B5823F099
:10342000405323F0030343F0805343F001038B50D8
:1034300023464FF4405143F23C02FFF7AAFF134AE0
:10344000134913684FF49B7043F080531360536823
:1034500043F0805353602A680E4BD150FDF740F97A
:10346000304606B0BDE8F0813C8F0000A493000018
:10347000988E0000C2900000BE8E0000000180A364
:10348000B88E0000280180A3000080A3000880A35C
:10349000FF000080300180A370B501460468C06859
:1034A00086B0B8B1FFF7D4FA0C4B014660791E68BC
:1034B000E27823790090607A019004F10C00029088
:1034C000658A35440395E08A304404904FF0FF301C
:1034D000FFF79AFB002006B070BD00BFE893000024
:1034E00008B50448FFF7D8FF40F28110FDF7F8F85F
:1034F000002008BD8090000008B54FF4B870FDF7BB
:10350000EFF80248FFF7C8FF002008BD3890000020
:1035100008B54FF4B070FDF7E3F80248FFF7BCFFC1
:10352000002008BD1490000008B54FF4A870FDF706
:10353000D7F80248FFF7B0FF002008BDF08F000069
:103540002DE9F0412E4F2F4E97F8745086B0736AD4
:103550002846984780464FF49070FDF7C1F806233F
:103560000093294B00210293284B01910393284B90
:103570004FF0FF3004930A460B46FFF745FB044625
:10358000002838D107F16C00FFF786FF4FF49170E7
:10359000FDF7A6F873692846D8F824709847B8470D
:1035A00040F22310FDF79CF81A4A1B4813684FF4A9
:1035B000405123F0405323F0030343F0805343F082
:1035C0000103136043F244022346FFF7E2FE134A6D
:1035D00040F22710136843F080531360536843F0A0
:1035E00080535360136D43F0010313650C4A0D4B78
:1035F0001A60FDF775F8204606B0BDE8F08100BFFF
:103600003C8F0000A4930000BC8E0000FE8E0000E2
:103610006F8E0000280190A6000090A6000890A6DA
:10362000FF000080300190A62DE9F043314F324E6B
:1036300097F8505087B0736A2846984781464FF4F0
:103640008870FDF74DF82D4B002102932C4B4FF065
:10365000030803932B4BCDF80080049301914FF0A6
:10366000FF300A460B46FFF7CFFA044600283DD14B
:10367000254B01221A6007F14800C3F80480FFF7C8
:103680000BFF4FF48970FDF72BF873692846D9F8C2
:1036900024709847B84740F21310FDF721F81B4AF1
:1036A0001B4813684FF4405123F0405323F00303A9
:1036B00043F0805343F00103136043F24402234676
:1036C000FFF767FE134A4FF48B70136843F0805383
:1036D0001360536843F080535360136D43F001034C
:1036E00013650D4A0D4B1A60FCF7FAFF204607B030
:1036F000BDE8F0833C8F0000A49300009A8E000088
:10370000F88E00006C8E0000001880A6280180A6AC
:10371000000080A6000880A6FF000080300180A67F
:10372000036823F04052084B22F003020B4013437E
:103730000360064B994206D050F8083C002B02DA91
:103740000838FFF71EBE704703000030010000106C
:10375000F0B53B4C4FF0000EBDF81C60BDF820509A
:10376000099FC4F800E0DFF80CE1CEF80060CEF865
:103770000460CEF80860CEF80C60324E0EF10C0EEC
:1037800035607560B560F560050445F0905545F409
:103790008055A6F5987635602B4D2C4EA5F5017514
:1037A000C5F804620C3EC5F808622026C5F8F06131
:1037B00017B1274E2E6000E02F60012841F4905190
:1037C00008BF0904234D244E0CBF41F48451090461
:1037D0002E6008BF41F01C0105F104051F4815BF0C
:1037E00041F484512960002600211CBF41F01C01D6
:1037F0002E6042F490520160194D1A4853B11A4993
:1038000012041B0442F48152194342F0140229604D
:10381000026007E0120442F48152134B42F014029A
:103820002A600360114B124A1A60A2F580329A6036
:1038300040F2712323602368DB05FCD4F0BD00BF98
:10384000003CA8A5403FA8A5143EA8A51018031247
:1038500000000280143CA8A500000780283CA8A511
:103860001C3CA8A5203CA8A534180012243CA8A5FF
:1038700000000480303FA8A5054B186003F58013B5
:10388000186003F58013186003F580131860704703
:10389000080100A608B50748FFF773FD0648FFF7C3
:1038A00070FD0648FFF76DFDBDE808400448FFF7CE
:1038B00068BD00BF000100A6000110A6000120A6FF
:1038C000000130A62DE9F0410F46364E364D374CFB
:1038D000002832D0C0F30222962353434FF02642F1
:1038E000136002F58012136002F580121360DFF896
:1038F000C48002F580121360D8F800202C4B1340CE
:1039000043F000431843C8F800003060286020608E
:10391000FFF7C0FFD8F8003043F01003C8F80030BC
:10392000336843F0100333602B6843F010032B60BF
:10393000236843F01003236014E01E4B1A6822F042
:1039400010021A60326822F0100232602A6822F0F7
:1039500010022A60226822F0100222601860306093
:1039600028602060144B154A19680A40BA4217D0E3
:103970001A68C7F3022022F010021A60962242430E
:103980000F4802600A4A0A403A4342F000421A6075
:103990001968094A8900FBD5136843F010031360C6
:1039A000BDE8F081000110A6000120A6000130A6AC
:1039B000F8C000FC000100A64001A8A5073FFF03D6
:1039C0000400A8A5054B064A103B1A6140F271227B
:1039D0001A601A68D205FCD4704700BF103CA8A535
:1039E000000002802DE9F04F05468BB001230893BB
:1039F0004C4B00221C680992E388E68A234433F882
:103A0000251003EB85035B88A0190793A678638ACA
:103A1000069104EB030E34F8038006FB05F3C15C4A
:103A2000C61873780231A04458F821700233BEF8EA
:103A3000021004EB830353F801B0A38AA94603EBF9
:103A4000C50354F803A0384B9A450DD1374B0320DA
:103A50005B6A9B8A2344D969354B01F5C341D3F88E
:103A600010C0283108ABE04738465946FFF72AFF17
:103A70005FB94FF47A730120029303930097019783
:103A80000497014605223B460AE00699B278F3788E
:103A90000291079900200391009001900490042165
:103AA000FFF756FE082D02DD05F1020903E0052DA2
:103AB000C8BF05F10109217A082901F1020301D9E2
:103AC000194602E0052988BF013158F8232046F243
:103AD0009053C2F309405843C2F30523B0FBF3F0FF
:103AE00002F00702D0404FF4FA6300F2CF70B0FB4F
:103AF000F3F05FFA89F280B2C9B20E4BFDF76AFAB1
:103B0000094B01219A459CBF012309930A4B186870
:103B1000002382680093946909AAA0470BB0BDE80E
:103B2000F08F00BFE8930000C8E40C003C8F000059
:103B3000A4930000AD870000D49300008140C943E6
:103B400010B50C4C824023680B480B401343236094
:103B500003680B401343036000F5801003680B40BB
:103B60001343036000F58010036819400A430260A4
:103B700010BD00BF000800A6000810A670B596266C
:103B800046439D0005F1254505F528052E60094DA4
:103B90005B015E5942F00042074C42EA014141EAB2
:103BA0000022344014435C515819BDE87040FFF7BF
:103BB000E8BB00BF2001A8A5F8C000FCF0B5414C4F
:103BC00087B04FF4A070FCF78BFD2368002B11DB4E
:103BD00000220123042040F21F11FFF7CFFF3A4AD1
:103BE000136823F0405323F0030343F0805343F062
:103BF00001031360354D40F24110FCF771FD2B6855
:103C0000002B11DB002203230D2040F23B11FFF7B4
:103C1000B5FF2F4A136823F0405323F0030343F00A
:103C2000805343F0010313602A4E4FF4A170FCF758
:103C300057FD3368002B10DB002204230820CD2120
:103C4000FFF79CFF244A136823F0405323F003033B
:103C500043F0805343F00103136040F24310FCF73C
:103C60003FFD092300931D4B002102931C4B019142
:103C700003931C4B4FF0FF3004930A460A23FEF7D0
:103C8000C3FF0746D8B91848FFF706FC40F24510B5
:103C9000FCF726FD2368154A43F0100323601368E0
:103CA00040F2471043F0100313602B6843F01003F9
:103CB0002B60336843F010033360FCF711FD384686
:103CC00007B0F0BD4001A8A54801A8A58001A8A59E
:103CD0008801A8A5A001A8A5A801A8A5C0900000DA
:103CE000D28E0000BF8E0000608F00006001A8A58A
:103CF0002DE9F04F05460668DFF89891B38AD9F8A8
:103D0000000099B0C3181093337A002707935C4BD7
:103D10004FF0010B11911B693946CDF858B0179738
:103D200004200B929847D9F80030728A119899189C
:103D300033F80280B1F802A0F28A294698449A44E6
:103D400013440893FEF784FE29460D900B98FEF766
:103D50007FFE0D9B0446BB4202DA4FF0FF306AE261
:103D60000028FADB474B5946186817AA8368009762
:103D7000D3F818C03B46E0473A4659461D20FFF7A6
:103D8000DDFE6B7A0E932B7A09933F4B09985B69A2
:103D90009847109B0C9003EBC4035A682B69D31807
:103DA0000A93B37803FB04F20F920F99089A525CBE
:103DB000023258F82270089A0A44527802325AF8AD
:103DC000222012920D9A5343089AD35CD9F800200E
:103DD000023358F82310F3882C4E134433F8240090
:103DE00003EB84035B8814901593119BB34205D9B0
:103DF0000B9BB34294BF0226012600E0022617B1B6
:103E000009B1012E09D002264FF001094FF0040A32
:103E1000DFF884804FF00A0B07E0DFF880804FF076
:103E200000094FF0050A4FF0060B194B03205B6A9F
:103E30009B8A1344144AD968D2F810C016AB0022EA
:103E4000E04740462946FEF703FE013885D4109B23
:103E5000082C03EBC000456805F55B4505F1BA0584
:103E600005DD079B0133DBB20793A31C06E0052C9D
:103E700016DD079B0133DBB20793631C109310E040
:103E8000D88D0000D4930000A4930000C7E40C0078
:103E90003C8F0000E893000008220800883C0E00D8
:103EA00010940C999F4BA04A1198904288BF1946D4
:103EB000A9420C9107D29D4B0998D3F810C029460E
:103EC0000E9A16ABE0470120FCF736FC594601225A
:103ED00000230798FCF75AFE0220FCF72DFC0F9BED
:103EE000022002331393139A089BDFF888B29B5C7D
:103EF0001193FFF7C1FCDBF80020002A02DA5846D4
:103F0000FFF73FFA8A4A0BF5801B9345F3D1119BCB
:103F100013F0FB0B01D0022E03D186480221FFF7DC
:103F2000FFFBBBF1010F02D0012E00D01FB9824868
:103F30000221FFF7F5FBBBF1020F03D17F48594681
:103F4000FFF7EEFB119B032B03D17D480221FFF706
:103F5000E7FB00230120009301934FF47A7331466D
:103F600052460293039304904B46FFF7F1FB754EC4
:103F70000320FCF7E1FB744A744BC6F80080D2F8CA
:103F800038C01B68724A9BB2117904200D22E047A9
:103F90000420FCF7D1FB0D9BB146A34203DC38465D
:103FA0001299FFF78FFC0520FCF7C6FB0C9BAB4278
:103FB0000AD90A9B09989D4238BF1D465B4B29468A
:103FC0001E690E9A16ABB0470620FCF7B5FB614B95
:103FD0001B681A68604B9A4200F02C81022C08DCA6
:103FE000524E03217368002098477368062003210E
:103FF00098470A9BDFF834819D4206D21946D8F8CB
:10400000106009980E9A16ABB0470720FCF794FB96
:104010000D9BA34203DD38461299FFF753FC08209D
:10402000FCF78AFB002207989DF840101346FCF726
:10403000ADFD0920FCF780FB77B94FF47A730120BE
:1040400002930393009701970490014605223B4693
:10405000FFF77EFB052635E0089B139A9E5C06F071
:10406000FB03012B0DD13D4F3A68002A09DB0420E8
:1040700040F21F110022FFF781FD3B6843F010035F
:104080003B60032E0DD1364F3B68002B09DB042328
:104090000820CD210022FFF771FD3B6843F010039B
:1040A0003B600F9A089B00201344149ADB7802921D
:1040B000159A009003920122049201900421324645
:1040C000FFF746FB274F3846FFF7D6FB36F00403D1
:1040D000184A05D024490968002901DA176001E06F
:1040E00022491160012B144A05D01C490968002996
:1040F00001DA1C4900E01D49022B11600F4B05D06D
:104100001B4A1268002A01DA164A00E0174A032EF9
:104110001A600B4B30D0124A1268002A2CDA114A6E
:104120002BE000BFC0C62D0040420F00A49300004A
:10413000000140A62801A8A54801A8A56801A8A5D6
:10414000A801A8A580000440D88D0000D8930000E5
:10415000308C0000BC890000054601154001A8A56F
:10416000A001A8A5010000102001A8A503000030AF
:104170006001A8A5000100A6304A1A600A20FCF7D9
:10418000DBFA0B9BC9F800300A9B9D4206D92C4BE9
:1041900009981D690A990E9A16ABA847294B2A4A15
:1041A0001B682A4D1179AE6B0D229BB20420B047DB
:1041B000274B0B9AD8F810709A4201BF254B264A1C
:1041C0005B6A126809BF9B8A00219B18D9694FF06E
:1041D000000204BF01F5C341283116AB0320B847E4
:1041E0000B20FCF7A9FA01211D200A46FFF7A6FCC7
:1041F0000C20FCF7A1FA022C114E07DD7368022196
:10420000002098477368062002219847104B0B9AAC
:104210009A420AD8114B0121186818AA8468002311
:1042200042F8041D0093A469A0470D4A2B6904209D
:1042300011789847002019B0BDE8F08F03000030D6
:10424000A4930000D8930000308C0000D88D0000AB
:10425000C8E40C003C8F0000E8930000D4930000F9
:10426000DC930000024A136843F0100313607047A8
:10427000000140A6094B05221A600122A3F5006344
:104280001A6003F5C013002203F5FF631A60044AA5
:10429000136843F010031360704700BF0818A8A507
:1042A0000001C0A50B4B05221A600122A3F5006393
:1042B0001A60A3F5FF2300220C3B1A60064A13681C
:1042C00043F01003136052F8203C43F0100342F80F
:1042D000203C70470C18A8A54001A0A50D4A012359
:1042E000136002F17F4202F5680208320421116076
:1042F000A2F10812136002F5C00203230432136016
:1043000002F58012136002F58012136002F580122C
:10431000136070470018C0A5024A136843F01003E9
:1043200013607047000181A5064B01221A60A2F1BB
:1043300001125A60044A0523136053609360D360EE
:10434000704700BF103FA8A5003FA8A5064B072255
:104350001A600022A3F608031A60044A136843F0A7
:1043600010031360704700BFFC18A8A5000101A04E
:104370002DE9F0414FF48070FCF7B2F9B54B4FF4E2
:104380001672B54D1A602B68B44AB54C1A40B54B3D
:10439000B549134340F29E722B60B44B1A602368F8
:1043A000AE4A1A40B24B13432360C868FEF750FB75
:1043B000071E01DA30BFFDE7AE4B1B68DA8A991899
:1043C0009A7807FB0212598A967892F803E052789D
:1043D00019444988023203EB8203032E58581DD03A
:1043E000052E01D0012E24D1C0F305239621594377
:1043F000A14ADFF8CCC21160DCF800209F491140CF
:1044000041F0004200F007010A4342EA0322C0F3F0
:10441000094342EA0343CCF800300AE0984B4FF4DA
:10442000966298491A600B688C4A1A40964B13435F
:104430000B60964B04221A6003F5B003032203F2CB
:10444000747393491A6002230B6001F580110C31DB
:104450000A6041F80C3C01F580110A6041F80C3CFF
:1044600001F580110A608B4A032E1360A2F52F021A
:10447000A2F104021360884BC3F800E0A3F50063C7
:104480001E600AD0052E01D0012E15D140F2011078
:10449000FCF726F9DFF8288205E04FF48170FCF77D
:1044A0001FF9DFF8E0814046FEF76BFFD8F80030D7
:1044B00043F01003C8F8003040F20310FCF710F985
:1044C0006548FEF75EFF4FF48270FCF709F9644817
:1044D000FEF757FF2B684FF0010843F010032B60E5
:1044E000236843F0100323606C4BC3F80080A3F5EE
:1044F0000063C3F80080FFF7B5FE40F20510FCF73B
:10450000EFF8FFF7CFFEFFF7B5FEFFF70DFFFFF760
:1045100003FFFFF71BFF4FF48370FCF7E1F8604ADD
:104520004FF040531360A2F500021360A2F5001291
:10453000136002F500221360A2F51C121360A2F1B1
:10454000B0621360574B40F20710C3F80080A3F528
:104550001C13C3F800800023136502F1B46202F556
:10456000E12210321360504B07221A60FCF7B8F8B2
:104570004E4B1B689B68DB6998473846FFF732FA59
:1045800040F20910FCF7ACF84948FFF775F9062E20
:1045900000F2C980DFE806F0041D3F98041D3F00CB
:1045A00044484549FFF7BCF82368002B0ADA434A20
:1045B000136823F0405323F0030343F0805343F088
:1045C000010313603E4B1B68002B80F2AC803D4A18
:1045D00016E02B68002B0ADA364A136823F04053A2
:1045E00023F0030343F0805343F001031360354885
:1045F0003149FFF795F82368002B80F294802F4A09
:10460000136823F0405323F0030343F0805343F037
:104610000103136087E02B68002B0ADA254A136830
:1046200023F0405323F0030343F0805343F001038E
:104630001360234B1B68002B0ADA224A136823F00D
:10464000405323F0030343F0805343F0010313600E
:104650001A4865E00000A8A52001A8A5F8C0007CC4
:104660006001A8A5000448813C8F00000800A8A5AF
:10467000000D9081E89300000400A8A5F8C000FC9C
:104680001000A8A5A001A8A50008CD809C10A8A591
:10469000041800A6041830A63418A8A50418A8A564
:1046A000000840A65008A8A51018A8A5D49300009B
:1046B000010000102801A8A5030000306801A8A58A
:1046C0004001A8A54801A8A52B68002B0ADA394AA1
:1046D000136823F0405323F0030343F0805343F067
:1046E00001031360344B1B68002B0ADA334A13684A
:1046F00023F0405323F0030343F0805343F00103BE
:1047000013602368002B0ADA2D4A136823F0405304
:1047100023F0030343F0805343F00103136029485F
:104720002949FEF7FDFF4FF48570FBF7D9FF032100
:104730000A461C20FFF702FA244A0123136002F5FF
:104740008012136002F58012136002F5801213606C
:104750001F4B204A40F20B10136002F580121360C9
:1047600002F58012136002F5801213601A4A13607A
:10477000136213641366C2F88030FBF7B1FF174B66
:104780001B689B7A23B1DA0242EA8332134301E0C9
:104790004DF60303124A4FF486701360FBF7A0FF37
:1047A000FFF79CFD40F20D10FBF79AFF0020BDE8DB
:1047B000F08100BF2801A8A54001A8A54801A8A52F
:1047C0006801A8A5A801A8A503000030500800A60C
:1047D000FF000080100100A63001A8A5B8890000E4
:1047E000000383A51A4B0A2270B51A80194B0B22BD
:1047F0001A80194B0C221A80184B0D221A80184B64
:10480000184A1D461360184A03F500611160002123
:10481000988A1E7A154A00EBC6008B505418285807
:104820002431B1F5B47FE06003F11803F0D1104BEF
:1048300010491B68D2F8942013F4700318BF20238A
:104840000B6009680C4B00200B44D36070BD00BFA7
:10485000F2930000F0930000EE930000F493000048
:1048600000940000E8930000F89300003C8F0000E3
:10487000100000A0B88E0000000180A370B50C4DA0
:104880000C4C2B680E469A68282303FB0040136AE1
:1048900000F10804408998472B6820F00C019B68C0
:1048A00060885B6A41EA86019847002070BD00BFBE
:1048B000D4930000FC900000002070470020704757
:1048C00010B5084B084A1B689968282358430B6A9F
:1048D0001418105A9847A378E2680340206900FB37
:1048E000032010BDD4930000FC900000F8B51A4BD3
:1048F00000241B689B68DB699847082C1AD0174B6B
:1049000020465B699847164A037A0668282101FB0E
:104910000321144B327AB08A1B6800EBC2021A449E
:104920000D695268CB682A44013AD31AB3FBF5F3F8
:104930000F193B7501340A2CDFD10024E0B2FFF7D8
:10494000BFFF074A282303FB04230134112C5860BE
:10495000F4D10020F8BD00BFD4930000248F0000E4
:10496000FC900000E8930000034B08461B681146CA
:104970009B685B6A184700BFD493000008B5044BDE
:1049800008461B689B681B6A9847C0B208BD00BFF9
:10499000D493000008B5064B06491B689A68282383
:1049A00003FB0010136A00899847C0F3811008BD0B
:1049B000D4930000FC900000024B282202FB003040
:1049C000704700BFFC900000044A0548136813F0CC
:1049D000807F044B08BF184610607047000382A612
:1049E000208F0801208F0800084B984205D8084BFB
:1049F00098428CBF1B20242000E01220054B1A682F
:104A0000520648BF40F0400018607047A0BB0D0040
:104A100000350C00000392A64DF60303044A054935
:104A200088428CBF18461046034B1860704700BF81
:104A30000420010000350C00000382A32DE9F04F93
:104A40008A4685B09B46AC4F01230393282303FB82
:104A50000073D968A0F103088A4528BF1B695FFA73
:104A600088F821BF03F1FF356D1A5544B5FBF3F506
:104A700034BF0025EDB2B8F1010F044600920CD806
:104A8000009BD7F84062F818D7F83C32721ED31A50
:104A90005344B3FBF6F380F8443228226243BB1838
:104AA00000985E681818B245057513D2002398184F
:104AB0003844007D58B185423FBFDFF83CE22825ED
:104AC00005FB04E52D693CBF05FB001A05460133D3
:104AD0000D2BECD1B24500F04C82282303FB04736C
:104AE0005B6A1BB1B24501D250469847A4F10F034F
:104AF000012B824E02D845F0C005E2E00E2C02D117
:104B000045F04005DDE0012C40F0CB807C497D4A3A
:104B100008681368007A894628B97B498A459CBF92
:104B200023F080731360794B1B681B79002B00F016
:104B3000A380774B5A6892455DD9764A92452ED923
:104B4000DFF8D891D9F800204AB33268682192681A
:104B50004FF48E70526A0193904732685E219268DA
:104B600040F24310526A904743F2D400019B5B68C5
:104B7000C3F5672303F56F63B3FBF0F0013000F07A
:104B800015FA5F4A336812689B6811785B6A40F2D5
:104B9000391001F0FB0198470023C9F800305C4B45
:104BA0005A685D4B9A4209D8013B9A4506D9336849
:104BB0004FF48E709B6888215B6A9847574B1B683F
:104BC000002B40F0EC80564AAAF5C331A03991423F
:104BD00038BF114646F2A812A1F586216FF40E7C6B
:104BE0006144B1FBF2F1336840F243109B6841F03D
:104BF00040015B6A53E0444B9A4211D901339A4514
:104C000000F2CD80336888219B684FF48E705B6A18
:104C10009847336840F243109B685E215B6A98476F
:104C20003C4B9A4500F2BB803C4A1368002B40F095
:104C3000B680336868219B684FF48E705B6A01927E
:104C4000984743F2D400324B5B68A3F56723A3F582
:104C50006F63B3FBF0F0013000F0A8F93368D9F8C6
:104C600000109B6809785B6A40F2391041F01C0122
:104C700098470123019A22E02A4B9A4540F28F80FF
:104C8000234A52689A4200F28A8040F2391033680F
:104C9000D9F800209B6811785B6A01F0E70198471A
:104CA0007DE0022C0DD116491F4A09681368497A24
:104CB000002974D11D498A4571D823F0400313603F
:104CC0006DE0B8F1010F33D80D4B1B685978D7F858
:104CD00034329A4563D94CF250334909594301F5AE
:104CE000122101F5F861514538BF5146009A03ABD6
:104CF0000E20FFF7A3FE52E0FC900000D4930000CA
:104D0000B8890000000382A62F8C1100BC89000026
:104D100024910000EF7E0E00308C1100CC93000037
:104D200090051000E0C81000000392A68F05100047
:104D30000B2C34D1914B1B6893F80390C9F3C1033A
:104D4000022B2CD18E4B5B689A4528D9336840F2F0
:104D50004B109B681B6A98474CF2503E336800F03A
:104D6000C00298684FEA59130EFB03FEAAF54341AF
:104D70000EF51223503903F5F8638B4238BF0B460A
:104D800046F2A811A3F586236FF40E7E7344B3FB9D
:104D9000F1F1D0F82490114340F24B10C8474FF086
:104DA000280909FB04F937F8091007EB09037548CE
:104DB00045EA012100220193FBF70AFA326837F82D
:104DC000090092682946526A9047019BDBF800204F
:104DD0005B686AB143F2D40053458CBFCAEB03034E
:104DE000C3EB0A03B3FBF0F0013000F0DFF80EE094
:104DF00043F2D40253458BBFCAEB0300C3EB0A0353
:104E0000B0FBF2F3B3FBF2F30133CBF80030012C2B
:104E100041D15A495C4A08681368007A28B95B484E
:104E2000824584BF43F080731360594B1B681B7924
:104E30000BB3584B5B689A4580F08C80564B1B68CF
:104E4000002B40F08780554AAAF5C331A039914222
:104E500038BF114646F2A8126FF40E70A1F58621F4
:104E60000144B1FBF2F1336840F243109B6841F01A
:104E700040015B6A0DE04A4B9A456BD8454A52683F
:104E80009A4267D940F2391033680A689B681178F2
:104E90005B6A98475EE0022C0DD13849414A0968A7
:104EA0001368497A002955D13F498A4552D943F0C0
:104EB000400313604EE0B8F1010F17D82F4B1B6869
:104EC0005978D7F834329A4544D24CF250334909D4
:104ED000594301F5122101F5F861514538BF51469A
:104EE000009A03AB0E20FFF7A9FD33E00B2C31D164
:104EF000224B1B68DD78C5F3C103022B2AD1204B5E
:104F00005B689A4526D2336840F24B109B686D0966
:104F10001B6A98474CF250326A43336800F0C00E67
:104F2000AAF54341986802F51223503903F5F86356
:104F30008B4238BF0B4646F2A8116FF40E72A3F5F0
:104F400086231344B3FBF1F1426A4EEA010140F2B9
:104F50004B109047282303FB04735A6A22B15B6805
:104F60009A4501D950469047282303FB0474C4F89E
:104F700004A0002005B0BDE8F08F00BFB889000094
:104F8000B4920000ED870000000382A62F8C110070
:104F9000BC89000024910000CC9300009005100013
:104FA000E0C81000000392A68F0510001A2250439B
:104FB000064B074A0021196010601A68054A116003
:104FC00001221A601A68D203FCD570470000014024
:104FD0000400014008000140706C75675F73740045
:104FE0006175746F63616C00645F696E0074780052
:104FF0000F0F17171B1B1D1D1E1E27272B2B2D2DBB
:105000002E2E33333535363639393A3A3C3C47471C
:105010004B4B4D4D4E4E53535555565659595A5A62
:105020005C5C63636565666669696A6A6C6C71710C
:105030007878F0F0727274741B1B1D1D0F0F171718
:105040002B2B2D2D1E1E2727353536362E2E33338E
:105050003C3C474739393A3A4E4E53534B4B4D4DF2
:1050600059595A5A55555656656566665C5C636370
:105070006C6C717169696A6A7878F0F07272747434
:1050800000000000F000FC00E405F005C807CC07B4
:10509000D007D407D807DC07E007E407E807F007E4
:1050A000F407F807FC070008040808080C081008B3
:1050B000C007C4072008240828082C083008340832
:1050C00038083C0840085008540858085C08600834
:1050D000640868086C0870081408180880088408B8
:1050E00088088C089008940898089C08A008B008C4
:1050F000B408B808BC08C008C408C808CC08D00860
:10510000E008E408E808EC08F008F408F808FC08EF
:1051100000091009140918091C0920092409280983
:105120002C093009940698067C0080008400000059
:105130006C00000000000000000483A63412000090
:10514000000000000000000000000000000000005F
:1051500058FC190000020300000093A6341200005E
:10516000000000000000000000000000000000003F
:105170004811100000030200000883A3341200004D
:10518000000000000000000000000000000000001F
:10519000D054080000040900000038A634120000B2
:1051A00000000000000000000000000000000000FF
:1051B000D05F1B0000000900E09A0000F89A000090
:1051C000713D0000413800003D3800007566000068
:1051D000000000005555EEEE11EE22DD44BB88774D
:1051E00011EE22DD44BB88770001000100010001BF
:1051F00000010001000100010000000000000000AB
:10520000000000000000000000000000000000009E
:10521000000000000000000000000000000000008E
:10522000000000000000000000000000000000007E
:10523000000000000000000000000000000000006E
:10524000000000000000000000000000000000005E
:10525000000000000000000000000000000000004E
:10526000000000000000000000000000000000003E
:10527000000000000000000000000000000000002E
:10528000000000000000000000000000000000001E
:10529000000000000000000000000000000000000E
:1052A00000000000000000000000000000000000FE
:1052B00000000000000000000000000000000000EE
:1052C00000000000000000000000000000000000DE
:1052D00000000000000000000000000000000000CE
:1052E00000000000000000000000000000000000BE
:1052F00000000000000000000000000000000000AE
:10530000000000000000000000000000000000009D
:105310000000000000000000000103000001011077
:105320000001010001000000000000000000010178
:105330000102010F0000000000000000000000005A
:10534000000000000000000000000000000000005D
:10535000000000000000000000000000000000004D
:10536000000000000000000000000000000000003D
:10537000000000000000000000000000000000002D
:10538000000000000000000000000000000000001D
:10539000000000000000000000000000000000000D
:1053A00000000000000000000000000000000000FD
:1053B00000000000000000000000000000000000ED
:1053C00000000000000000000000000000000000DD
:1053D00000000000000000000000000000000000CD
:1053E00000000000000000000000000000000000BD
:1053F00000000000000000000000000000000000AD
:10540000000000000000000000000000000000009C
:10541000000000000000000000000000000000008C
:10542000000000000000000000000000000000007C
:105430000000000000020201000000010101000064
:1054400000000000050505050505050518183030A4
:105450000808101140101010080100000E08040484
:10546000000202020003030300040404000202021B
:10547000000303030004040401FF00000001010015
:10548000000001010000000003030000040101000E
:10549000000000000000000000000000000000000C
:1054A00000000000000000000000000000000000FC
:1054B00000000000000000000000000000000000EC
:1054C00000000000000000000000000000000000DC
:1054D00000000000000000000000000000000000CC
:1054E00000000000000000000000000000000000BC
:1054F00000000000000000000000000000000000AC
:10550000000000000000000000000000000000009B
:10551000000000000000000000000000000000008B
:10552000000000000000000000000000000000007B
:10553000000000000000000000000000000000006B
:10554000000005A6000015A6000025A6000035A64F
:105550000040A6A519530000D9510000C152000017
:105560000000000000000000014E0000454E000059
:10557000814E0000C94D000000000000B54E000043
:105580000D4F0000000000000000000000000000BF
:105590000000000099480000415000006D500000DC
:1055A00000000000D14B00000D4900000000000089
:1055B00000000000000000000000000000000000EB
:1055C00000000000000003A6000013A6000023A6B0
:1055D000000033A60080A6A5D15C0000B55D0000E8
:1055E000755B000015590000295B00009D58000004
:1055F000195B0000095B000015580000AD57000062
:105600000000000059580000D95800005956000009
:105610005D5E000009570000C15E00003D5F0000B4
:10562000B15F0000D9590000595900003D570000F2
:10563000E3660000E7660000EB6600001967000003
:1056400015690000CD680000E967000021670000CF
:105650000D67000011670000156700007169000008
:1056600051670000EF660000F566000001070701C2
:105670000707030103000000801A06000000010074
:10568000AA110400000002000071020000000400E2
:10569000A08601000000070080A380A63C10A8A5FA
:1056A0003C18A8A500000000000190A60C8F000087
:1056B000001090A6030100002000000090A6030146
:1056C00001020100020000000000010701010707BC
:1056D0000707841050100010BC1008114010A010D3
:1056E000B810F410101084180018C4180C194018C1
:1056F000A818C018FC18101808181018141810183A
:1057000018180C18081800180418000008220800BF
:1057100000000100041104000000030082080200E0
:10572000000007004D6A00000000000000000000BB
:10573000696B0000E5690000D1690000000000000D
:10574000C490000000000000000000000000000005
:10575000F17400000000000000000000717B0000F8
:105760000000000000000000030100000000000035
:105770000000000000000000000000000000000029
:10578000BD73000000000000A490000001020000B2
:105790000000000000000000000000000000000009
:1057A00000000000296E0000000000009C8E000038
:1057B00002030000000000000000000000000000E4
:1057C0000000000000000000416D0000000000002B
:1057D000E090000005040000000000000000000050
:1057E000000000000000000000000000AD6B0000A1
:1057F00000000000000000000305000000000000A1
:105800000000000000000000000000000000000098
:10581000296D0000000000000000000004060000E8
:105820000000000000000000000000000000000078
:1058300000000000116D00000000000000000000EA
:10584000040700000000000000000000000000004D
:105850000000000000000000F96C000000000000E3
:10586000000000000508000000000000000000002B
:105870000000000000000000000000000000000028
:1058800000000000000000000B0900000000000004
:105890000000000000000000000000000000000008
:1058A000E16C00003810A8A53818A8A50000000079
:1058B000000180A60C8F0000001080A603010000EC
:1058C000A8A504180000000000000000000000006F
:1058D00000000000000000000000000000010000C7
:1058E000000000008018A8A50000000000000000D3
:1058F000788E0000001080A3040100001A01FF0050
:105900000000000019011901E09304006A1800006A
:105910000000000000000000000000000000000087
:10592000000000001C01FF00000000001B011B0123
:10593000E09304006A18000000000000000000006E
:105940000000000000000000C98100001E01FF00EF
:10595000000000001D011D01E09304006A18000012
:105960000000000000000000000000000000000037
:10597000E98100002001FF00000000001F011F015D
:10598000E09304006A18000000000000000000001E
:105990000000000000000000000000002201FF00E5
:1059A0000000000021012101E09304006A180000BA
:1059B00000000000000000000000000000000000E7
:1059C000000000002401FF0000000000230123016B
:1059D000E09304006A1800000000000000000000CE
:1059E0000000000000000000198200002701FF00F5
:1059F0000000000026012601E09304006A18000060
:105A00000000000000000000000000000000000096
:105A1000000000002901FF0000000000280128010B
:105A2000E09304006A18000000000000000000007D
:105A30000000000000000000000000002B01FF003B
:105A4000000000002A012A01E09304006A18000007
:105A50000000000000000000000000000000000046
:105A6000000000002D01FF00000000002C012C01AF
:105A7000E09304006A18000000000000000000002D
:105A80000000000000000000000000002F01FF00E7
:105A9000000000002E012E01804F1200D4300000C3
:105AA00000000000000000000000000000000000F6
:105AB000000000003101FF00000000003001300153
:105AC000E09304006A1800000000000000000000DD
:105AD00000000000000000000000000034017F0012
:105AE000000000003301330140AC2700D430000037
:105AF00000000000000000000000000000000000A6
:105B0000000000003F013F00000000003F013F0196
:105B100060AE0A00A8610000000000000000000064
:105B200000000000000000000000000044013F00F1
:105B30000000000044014401E0930400A86100005B
:105B40000000000000000000000000000000000055
:105B50000000000048013F0000000000480148012B
:105B6000801A0600D4300000000000000000000091
:105B700000000000000000000000000049013F009C
:105B80000000000049014901801A0600D4300000DD
:105B90000000000000000000000000000000000005
:105BA00000000000ED8000007D800000B980000052
:105BB000BD8000003D820000C18000007D810000AA
:105BC0006981000095810000B9810000010000009A
:105BD00000000000000000000000000000000000C5
:105BE00000000000000000000000000000000000B5
:105BF00000000000000000000000000000000000A5
:00000001FF
